:103E99000F560F4B0F3F0F330F260F180F0A0EFB4C
:103EA9000EEB0EDA0EC90EB70EA40E900E7B0E6540
:103EB9000E4F0E370E1F0E050DEB0DD00DB40D96DE
:103EC9000D780D590D390D180CF50CD20CAE0C8965
:103ED9000C630C3D0C150BED0BC30B990B6F0B43CE
:103EE9000B170AEB0ABD0A900A620A330A0409D5BC
:103EF90009A609760946091708E708B7088708587F
:103F0900082807F907CA079C076E0740071306E642
:103F190006BA068E06630639060F05E605BD059540
:103F2900056E0548052304FE04DA04B704940473F6
:103F390004520432041303F403D603B9039D038224
:103F49000367034D0334031B030302EC02D602C0CB
:103F590002AA02960282026E025C02490238022615
:103F69000216020601F601E701D801CA01BC01AF38
:103F790001A201960189017E01720167015D015269
:103F89000149013F0136012C0124011B0113010BD9
:103F9900010300FC00F500EE00E700E000DA00D4C0
:103FA90000CE00C800C300BD00B800B300AE00A930
:103FB90000A400A0009C00970093008F008C00884B
:103FC90000840081007D007A007700740071006E22
:103FD900006B0068006600630061005E005C0059C8
:103FE9000057005500530051004F004D004B004948
:103FF9000047004600440042004100010C01010550
:1040090002011E030A96040132050505060064072C
:10401900010108000009015A0E01010F00011200F7
:104029006413010114013C1501FA1664FA17FFFF24
:104039001D00072000072400022701012F013C3041
:10404900030332010335FFFF3603073C32963DFF78
:10405900FF180002191E461A00021B00022D32C861
:064069002E0001FAFAFA34
:10004800900787E0FEA3E0FF7457BE0010D39F40DF
:100058000C90400312001EE493F5998012900787D4
:10006800E0FEA3E0FF90400312001EE493F5999090
:10007800078712000E900787E0FEA3E0FF746C6FFD
:100088004E700375130022900073E0B401087402E7
:10009800900073F0D21390013BE090002AF0900199
:1000A8003CE090002BF090013DE090002CF0A20D78
:1000B800B3401690013BE0700C90013CE070069054
:1000C800013DE060028002C20D90013BE0B4300FB8
:1000D80090013CE0B4470890013DE0643B60028039
:1000E80004D20E8002C20EE558B401028003020257
:1000F80011900058E0F568900063E0F56A9000649C
:10010800E0F56B900075E0F56C90007BE0900029BD
:10011800F090007DE0F56790007EE0F56990008141
:10012800E0F566900082E0F565900091E09000416E
:10013800F0900092E0900042F0900093E09000432D
:10014800F0900094E0900044F0900095E090004515
:10015800F0900096E0900046F0900097E0900047FD
:10016800F0900098E0900048F090009AE0900033FA
:10017800F090009BE0900034F090009CE0900035F7
:10018800F090009DE0900036F090007AE0B40117FE
:1001980090000A740FF0A374FFF090000CE4F0A331
:1001A800F0740290007AF090007AE0B4035990005D
:1001B8000CE0FEA3E0FF90000AE0FCA3E0FD1200C3
:1001C8000374101241CF74081241C1EF900026F059
:1001D800EF700674FF900026F0740090007AF0909B
:1001E800000BE0900027F090000AE0900028F090C3
:1001F8000026E090078AF0900027E090078BF090A7
:100208000028E090078CF0803F900082E07006752F
:100218005801756500A20DB3402E90013BE0900097
:100228002AF090013CE090002BF090013DE0900016
:100238002CF090002AE0700C90002BE070069000E3
:100248002CE060028002C20DE5687003756802E563
:100258006A7003756A027E897FE7E5688E048F05F8
:10026800FF1241B18C398D3AE56B75F0FAA4FFAEF7
:10027800F0E56A8E048F05FF1241B18C3D8D3E90EA
:100288000050E0F56290004DE0FE90006AE0B5068F
:100298001890004CE0FE900069E0B5060C90004B09
:1002A800E0FE90005AE06E606F90006AE070069081
:1002B8000069E06006740090005AF090006AE0B4AB
:1002C80002089000497401F08005900049E4F0901C
:1002D8000069E0B4020890004A7401F080059000BB
:1002E8004AE4F0900069E0600690004AE06002800D
:1002F800057562048003756205E559B55802D21385
:10030800900069E090004CF090006AE090004DF099
:1003180090005AE090004BF0740090009FF0740138
:100328009000A0F074019000A1F074019000A2F078
:1003380074009000A3F074009000A4F07400900082
:10034800A5F074009000A6F074019000A7F0740165
:100358009000A8F074019000A9F074009000AAF031
:1003680074009000ABF074009000ACF07400900042
:10037800ADF074019000AEF074019000AFF074011C
:100388009000B0F074009000B1F074009000B2F0EA
:1003980074009000B3F07400900363F0740190034C
:1003A80064F07401900365F07401900366F07400C2
:1003B800900367F07400900368F07400900369F08C
:1003C80074019003A3F074009003A4F074019003E7
:1003D800A5F074019003A6F074009003A7F07400D0
:1003E8009003A8F074009003A9F074009003E3F060
:1003F80074009003E4F074019003E5F07401900335
:10040800E6F074009003E7F074009003E8F07400DD
:100418009003E9F07400900423F07400900424F031
:100428007401900425F07400900426F07400900480
:1004380027F07400900428F07400900429F07400E8
:10044800900463F07401900464F07400900465F003
:100458007401900466F07400900467F074009004CE
:1004680068F07400900469F022E5B554F7F5B5E535
:10047800B554FDF5B5C2A2C2A1C292C207E5B554F2
:10048800FBF5B5755105E55104F552900050E0F5BE
:1004980062900025E4F0C20A90004EE4F0E5B554FD
:1004A800FEF5B5C28E758D00758B00754C007526EE
:1004B80000752500D28E22750A00750900AE09AFB5
:1004C8000A7457BE00039F500302057C9040031234
:1004D800001EE49390004F1241E70FBF00010EE0A9
:1004E800FC90400312001EECFEE493FFEEC39F5005
:1004F80026AE09AF0A0FBF00010E90400312001E7E
:10050800AE09AF0AE493FC90400312001EE49390F6
:10051800004F1241E7ECF0AE09AF0A904003120019
:100528001EE49390004F1241E7E0FC904005120052
:100538001EECFCE493FDECD39D401990400512009D
:100548001EE493FC90400312001EE49390004F12A7
:1005580041E7ECF0AE09AF0A74022FFF50010E8E8E
:10056800098F0A780A740126F6500418E436F64012
:10057800030204C522750A00750900AE09AF0A74A2
:1005880015BE00039F500302064A90405A12001EEF
:10059800E49390004F1241E70FBF00010EE0FC907A
:1005A800405A12001EECFEE493FFEEC39F5026AEA5
:1005B80009AF0A0FBF00010E90405A12001EAE0983
:1005C800AF0AE493FC90405A12001EE49390004F47
:1005D8001241E7ECF0AE09AF0A90405A12001EE44F
:1005E8009390004F1241E7E0FC90405C12001EEC33
:1005F800FCE493FDECD39D401990405C12001EE48E
:1006080093FC90405A12001EE49390004F1241E769
:10061800ECF0AE09AF0A740F6F4E7006750A1575C7
:100628000900AE09AF0A74022FFF50010E8E098F20
:100638000A780A740126F6500418E436F6400302D4
:10064800058322054D22054C22054EC2CF2290F883
:1006580000E4936406600280FE75840175A7007546
:10066800FF80900789E4F075C91075A70F75A1C7B9
:1006780075A70075D90075CEFF75A70F75F1FE75C2
:10068800F2FF75F33775F47875A4BA75A5FF75A6EA
:100698000775AE0075AFFF75D48175D5FF75D6FFA8
:1006A80075D7FFC295C296C297C2A0E5B554BFF5EB
:1006B800B5C20FC210C211C212120471E5B554DFDF
:1006C800F5B5E5B554EFF5B5E5B5547FF5B5E5B540
:1006D80054F7F5B5E5B554FDF5B575A70075A20154
:1006E80075A14775F80975BC0175BE0475BD6C75B3
:1006F800BE0775BDA075BE0875BD0175BC0075BB8C
:100708001875BC2075BA0875E88075D11375A70FE0
:1007180075E10575E20075C7407597007597807497
:100728000A1241A17597C0E5975420700280F875A8
:100738008F0275A700D2AF75980075A90C75A70F21
:1007480075AB4375ADFB75AC1E75A7007589117542
:100758008E00758C00758A00D2A9D28C758D0075B3
:100768008B00D2ABD28E75CD0075CC0075CA0075E2
:10077800CB00D2ADC2CFD2CA7591047592007593E1
:10078800CD75EF0675D94075CF01900787E4F0A3C2
:10079800F0751300751400C299D20DC214120471B9
:1007A80074C8F5187517001227C875A70FE5FB90D0
:1007B800001AF0E5FA90001BF0E5F990001CF075BE
:1007C800A70090F800E493F5081228FF122E39903C
:1007D800078AE0900026F090078BE0900027F090C1
:1007E800078CE0900028F090078DE0900029F090A9
:1007F800078EE0F56890078FE0F56A900790E0F5BE
:100808006B900791E0F56C900792E0F5679007937D
:10081800E0F569900794E0F566900795E0F5659036
:100828000796E090002AF0900797E090002BF09050
:100838000798E090002CF0900799E0900041F09024
:10084800079AE0900042F090079BE0900043F090F8
:10085800079CE0900044F090079DE0900045F090E0
:10086800079EE0900046F090079FE0900047F090C8
:1008780007A0E0900048F09007A1E0900033F090C6
:1008880007A2E0900034F09007A3E0900035F090C4
:1008980007A4E0900036F07400900083F090013BCC
:1008A800E0700C90013CE0700690013DE060028031
:1008B80004C20D8002D20D90F807E493900021F055
:1008C800900021E0440A900021F0900021E054FEBD
:1008D800900021F07406900012F07402900013F05A
:1008E80090F802E493900014F07403900015F074EB
:1008F80003900016F07413900017F0740590001818
:10090800F07405900019F090F804E49390001DF03D
:10091800740090001EF090F805E49390001FF0908A
:10092800F806E493900020F074FF900022F0744AD7
:10093800900126F07461900127F07474900128F0FA
:100948007463900129F0746F90012AF0742090016B
:100958002BF0745290012CF0744590012DF07435F1
:1009680090012EF0745290012FF07430900130F005
:100978007435900131F07441900132F07420900187
:1009880033F07435900134F090007BE0D39401404B
:1009980006740090007BF075580175590174039036
:1009A800004CF012008F1204BF12057D1227F4E5E7
:1009B800B554FEF5B5900025E4F0900787E4F0A360
:1009C800F0752400752300754800752A0075290004
:1009D800754900753200753100754A007554007507
:1009E8005500755A0075510575520175343C7533BB
:1009F800007574007573007575CD755600755700D0
:100A0800754300754400754500754600755B0075B3
:100A18004700754200754100900006E4F0A3F0908D
:100A28000008E4F0A3F075600075610090000E7492
:100A3800FDF0A374E8F0900023E4F07464900024BF
:100A4800F0C200D201C202D203754D00756F00C218
:100A580094C293C287C290C291C2137E017F009054
:100A68000028E01241CF900027E02FFF50010E90A0
:100A7800000AEEF0A3EFF0900026E0700674FF90F5
:100A88000026F090000AE0FEA3E0FFEFD394FFEE0B
:100A9800940F400790000AE4F0A3F07400900072ED
:100AA800F0740090007AF07400900083F074009065
:100AB800008EF074009000B5F0E569700375690464
:100AC800743A90074FF074FD900750F0900415E0C9
:100AD800900455F0D2B0D2B7D2A7D2A6D2B1D2A341
:100AE800C207A2B6B39204A2B3B39205D29CD2ECC9
:100AF80075CF01A298B34005C29812319DE51360E5
:100B080006A299B3B340028005C29912370DE514C5
:100B180064016005E514B4040280D5E54DD394055D
:100B2800400CE55AC394C85002055A754D00E57546
:100B3800C394E95023787312003FAE73AF749000EA
:100B48008CE075F064A4FDACF0EFD39DEE9C4008FA
:100B58000575757400757300C28E7E047F00E54CC0
:100B68001241CFE58D75F004A4FDACF0EF2DFDEE3C
:100B78003CFCE58B75F04084FF7E00ED2FFFEC3EDA
:100B8800FE8E258F26D28EA2B6300401B350030202
:100B98000CD4A2B6300401B35003020CD4A2B64060
:100BA800670554A214400575FFA0D214E5B54401A9
:100BB800F5B5900024E4F0E554D3956840487C8965
:100BC8007DE7AE25AF2612406F8E238F24E5482F90
:100BD800FF50010E74011241C18E238F24852448D1
:100BE800755401C28E758D00758B00754C00D28EC0
:100BF8007403BE00039F50069000257401F0E5437E
:100C0800B40603754300D204A2B6B35003020CD451
:100C1800C20490006CE0601812384EA200B340087D
:100C2800E5B54408F5B58006E5B554F7F5B5800295
:100C3800C20090006FE060181239A3A202B3400806
:100C4800E5B54402F5B58006E5B554FDF5B5800671
:100C5800E5B554FDF5B5A207B34004D2878002C2BA
:100C68008790005AE06004D2908002C29090004AB7
:100C7800E0B40104D2948002C294900049E0B40127
:100C880004D2938002C293A20AB34004D291800294
:100C9800C291900018E0FE900014E0C39E400990B5
:100CA8000014E0D39408400974FB900023F0120468
:100CB8007190001DE0601590001DE0FE900017E0A7
:100CC8006E600974FE900023F0120471C2CA7E019E
:100CD8007F00E54E1241CFE5CD2FFF50010E8E2744
:100CE8008F28D2CAE567B4014890000EE0FCA3E063
:100CF800FDEFC39DEE9C4039B209E52A45296013F2
:100D0800A209B34008E5B54404F5B58006E5B55435
:100D1800FBF5B590000EE0FEA3E0FF900010E0FCAC
:100D2800A3E0FDEF2DFDEE3CFC90000EECF0A3EDF2
:100D3800F0A2B3300501B35003020E22A2B330056E
:100D480001B35003020E22A2B35003020E1B055535
:100D5800A214400575FFA0D214E5B54401F5B5907D
:100D68000024E4F0E555D3956A5003020E197CEA95
:100D78007D60AE27AF2812406F8E298F2AE56B124F
:100D880041CF74FF8E048F05FF1241B18C298D2A43
:100D9800E5492DFD50010C74018C068D071241C1E7
:100DA8008E298F2A852A49A20AB3401574641241F4
:100DB800CF900068E08E048F05FF1241B18C298D19
:100DC8002A75550190000EE0FEA3E0FFAC27AD2880
:100DD80012000390000EEEF0A3EFF0E569FF124158
:100DE800B1740AFF1241B190007CE08C068D0712A5
:100DF80041CF74148E048F05FF1241B1900010EC9E
:100E0800F0A3EDF0C2CA75CD0075CC00754E00D2C6
:100E1800CAD205A2B3B34002C205900025E0B401CE
:100E280007E556C394064003021442E56F9027A7CE
:100E3800F828287390005AE0C394024003020F90E8
:100E4800E551D394015003020F90E55175F040A489
:100E5800FFAEF090031312001EE0C395455018E54D
:100E68005175F040A4FFAEF090031212001EE0F599
:100E78002E752D00020F90E55175F040A4FFAEF0DD
:100E880090031112001EE0C395454003020F2CE5A4
:100E98005175F040A4FFAEF090031212001EE55108
:100EA80075F040A4FFAEF0E0FC90031012001EECB9
:100EB800FEE0FFEEC39FFEE5518E0475F040A4FFEF
:100EC800AEF090031112001EE0F40425458C008852
:100ED800F0A4FFAEF0E5518F048E0575F040A4FF35
:100EE800AEF090031312001EE55175F040A4FFAE5A
:100EF800F0E0FA90031112001EEAFEE0FFEEC39F35
:100F0800FECDCCCD8E071241B1E55175F040A4FF5E
:100F1800AEF090031012001EE02DFD50010C8C2D38
:100F28008D2E8064E55175F040A4FFAEF09003105B
:100F380012001EE55175F040A4FFAEF0E0FC9003EE
:100F48000F12001EECFEE0FFEEC39F8545F0A4FFE4
:100F5800AEF0E5518F048E0575F040A4FFAEF09019
:100F6800031112001EE0FECDCCCD8E071241B1E573
:100F78005175F040A4FFAEF090030F12001EE02D53
:100F8800FD50010C8C2D8D2E756F010214429000BE
:100F98005AE0C394024003021144900050E0D395F4
:100FA8005150030210ECE55175F040A4FFAEF090EB
:100FB800031912001EE0C395455018E55175F0401D
:100FC800A4FFAEF090031812001EE0F52C752B005C
:100FD8000210ECE55175F040A4FFAEF09003171233
:100FE800001EE0C395454003021088E55175F040A6
:100FF800A4FFAEF090031812001EE55175F040A44E
:10100800FFAEF0E0FC90031612001EECFEE0FFEECF
:10101800C39FFEE5518E0475F040A4FFAEF0900327
:101028001712001EE0F40425458C0088F0A4FFAEDA
:10103800F0E5518F048E0575F040A4FFAEF09003E3
:101048001912001EE55175F040A4FFAEF0E0FA90C9
:10105800031712001EEAFEE0FFEEC39FFECDCCCDC3
:101068008E071241B1E55175F040A4FFAEF0900330
:101078001612001EE02DFD50010C8C2B8D2C806467
:10108800E55175F040A4FFAEF090031612001EE57E
:101098005175F040A4FFAEF0E0FC90031512001E5D
:1010A800ECFEE0FFEEC39F8545F0A4FFAEF0E551EE
:1010B8008F048E0575F040A4FFAEF0900317120060
:1010C8001EE0FECDCCCD8E071241B1E55175F04042
:1010D800A4FFAEF090031512001EE02DFD50010C88
:1010E8008C2B8D2CE551B40123E562D39401401C6F
:1010F800E55604D395514014E545C39405500D9029
:101108000360E0A829B80006952A400280037551BB
:1011180002E551B56222900050E0D395514019E59F
:101128005175F040A4FFAEF090031812001EE0A81D
:1011380023B800069524400280020562756F0202FA
:10114800144290005AE0B4022AE55175F040A4FF19
:10115800AEF090031812001EE0F52C752B00E55137
:1011680075F040A4FFAEF090030F12001EE0F52EBC
:10117800752D0090005AE0B4030F900052E0F52C52
:10118800752B00752E00752D00756F03021442E54E
:101198005175F040A4FFAEF090032112001EE0C389
:1011A800955A400302126C900049E07036E551D31D
:1011B80094014029AE23AF24AC2DAD2EEDD39FEC86
:1011C8009E401AE55175F040A4FFAEF090031F123F
:1011D800001EE0A829B80005D3952A500280021500
:1011E800518034E551D394024029AE23AF24AC2D6D
:1011F800AD2EEDD39FEC9E401AE55175F040A4FF4B
:10120800AEF090031F12001EE0A829B80005D39580
:101218002A500280021551E551B55237E551C39560
:10122800625030E55604D395514028AE23AF24AC24
:101238002BAD2CEFD39DEE9C4019E55175F040A4E1
:10124800FFAEF090032012001EE0A829B800069512
:101258002A400280020551C292E55165526005C2DA
:1012680007755A00756F04021442E55175F040A4E1
:10127800FFAEF090031B12001EE0B40117E5517594
:10128800F040A4FFAEF090032112001EE0240AC330
:10129800955A4003021342753064752F00A207B3B4
:1012A800500B900061E02405C395454003021342AA
:1012B800E55175F040A4FFAEF090031E12001EE049
:1012C800C395454064E55175F040A4FFAEF0900326
:1012D8001D12001EE55175F040A4FFAEF0E0FC9031
:1012E800031C12001EECFEE0FFEEC39F8545F0A430
:1012F800FFAEF0E5518F048E0575F040A4FFAEF007
:1013080090031E12001EE0FECDCCCD8E071241B117
:10131800E55175F040A4FFAEF090031C12001EE0EA
:101328002DFD50010C8C2F8D30AE23AF24AC2FAD8A
:1013380030EFD39DEE9C4002D207756F0502144230
:10134800E551B4010990005AE0C394024003021425
:1013580016900359E0D3954550030214169003578D
:10136800E0C395455040900358E0FE900356E0F4E2
:10137800042EFE900357E0F40425458E0088F0A45F
:10138800FFAEF0900359E0FC900357E0F4042C8E74
:10139800048F05FF1241B1900356E02DFD50010C5A
:1013A8008C2B8D2C802C900356E0FE900355E0F496
:1013B800042E8545F0A4FFAEF0900357E08E048F0D
:1013C80005FF1241B1900355E02DFD50010C8C2B07
:1013D8008D2CE551C395625030E55604D3955140A4
:1013E80028AE23AF24AC2BAD2CEFD39DEE9C401937
:1013F800E55175F040A4FFAEF090032012001EE006
:10140800A829B80006952A40028003755102900069
:1014180049E0B40106E55164016002800375510298
:10142800E55165526005C207755A00E55AD3940A1A
:0A143800400590004EE4F0756F00CF
:1027A700020E3C020F9602114A02119702127202A0
:0227B7001348C5
:10144200900051E02402A823B80007D3952440025B
:10145200C207900025E0B4010990005AE0C394034A
:1014620040030215D6900049E0600302151FE551C2
:10147200D39401403A90004EE07034E55175F0404B
:10148200A4FFAEF090031512001EE0A823B8001FBF
:10149200D39524401AE55175F040A4FFAEF09003B5
:1014A2002012001EE0A829B80005D3952A50028018
:1014B200021551E551D39401402FE55175F040A436
:1014C200FFAEF090031312001EE0C39545501AE5DB
:1014D2005175F040A4FFAEF090031F12001EE0A869
:1014E20029B80005D3952A500280021551E551D33F
:1014F20094014022E55604C39551501AE55175F006
:1015020040A4FFAEF090031F12001EE0A829B8000D
:1015120005D3952A5002800215510215CBE551D30D
:101522009402403A90004EE07034E55175F040A4C8
:10153200FFAEF090031512001EE0A823B8001FD3DF
:101542009524401AE55175F040A4FFAEF0900320B7
:1015520012001EE0A829B80005D3952A5002800285
:101562001551E551D39402402FE55175F040A4FF87
:10157200AEF090031312001EE0C39545501AE551D8
:1015820075F040A4FFAEF090031F12001EE0A829E0
:10159200B80005D3952A500280021551E551D39423
:1015A200024022E55604C39551501AE55175F040A8
:1015B200A4FFAEF090031F12001EE0A829B8000598
:1015C200D3952A500280021551E55165526005C239
:1015D20007755A00900061E0D39545500990005577
:1015E200E0C395455002C20790005AE0700302180A
:1015F2003BA2A5B34008A2A4B34003021824AE350F
:10160200AF367441D39F749C9E4005783512003FDB
:10161200AE35AF36EFB48806EEB41302800302187B
:1016220001A2A550030216C490005AE0B4010B9027
:101632000050E0D395624002056290005AE0B40285
:1016420054E55175F040A4FFAEF090032112001E44
:10165200E0C3955A503F900050E0D395514021E5A8
:101662005604D395514019E55175F040A4FFAEF0F0
:1016720090031512001EE0A823B80006952440022C
:1016820080020551900050E0F562E5516552600517
:10169200C207755A0090005AE0B40326900050E049
:1016A200D395514008E55604D39551500280020566
:1016B20051900050E0F562E55165526005C2077530
:1016C2005A00A2A4500302180190005AE0B4016E1D
:1016D200900049E07035E551D394014029E55175F8
:1016E200F040A4FFAEF090031F12001EE0A829B83C
:1016F200000FD3952A400A1551755A008551628010
:101702000385516280037562018033E551D39402EF
:101712004029E55175F040A4FFAEF090031F12007E
:101722001EE0A829B8000FD3952A400A1551755A10
:1017320000855162800385516280037562029000C8
:101742005AE0D3940150030217F5E55175F040A415
:10175200FFAEF090032112001EE0C3955A4003022F
:1017620017F5900049E07041E551D394014034E50A
:101772005175F040A4FFAEF090031212001EE0A8D3
:1017820023B8001FD39524401AE55175F040A4FFF9
:10179200AEF090031F12001EE0A829B80005D395F1
:1017A2002A500280021551803FE551D39402403401
:1017B200E55175F040A4FFAEF090031212001EE056
:1017C200A823B8001FD39524401AE55175F040A410
:1017D200FFAEF090031F12001EE0A829B80005D347
:1017E200952A500280021551E55165526005C207E3
:1017F200755A00E556B4070405608003756000E57C
:1018020065B4010EAE35AF36EF64407005EE649CF0
:101812006002800EA2A54003755801A2A440037580
:101822005802A2A5B3B35006A2A4B3B340028006E5
:10183200753600753500021929A2A5B34008A2A485
:10184200B34003021915AE35AF367441D39F749C71
:101852009E4005783512003FAE35AF36EFB48806AC
:10186200EEB413028003021915A2A5406F9000691D
:10187200E0605A90004AE0B4010790004AE4F08028
:101882000690004A7401F090004AE0700575620407
:10189200800375620590004AE0B40104D29480028C
:1018A200C294E551B4051AE55175F040A4FFAEF0BB
:1018B20090031F12001EE0A829B80005D3952A50F4
:1018C200028008755104C207755A008003756205CB
:1018D200E556B4070405608003756000A2A4403396
:1018E20090006AE06021900049E0B401079000494D
:1018F200E4F080069000497401F0900049E0B401E0
:1019020004D2938002C293E556B4070405608003B3
:10191200756000A2A5B3B35006A2A4B3B34002807F
:1019220006753600753500E55865596006900083E6
:10193200E06003021AB1C29C751400751300C2CA9A
:10194200E5589027B9F82828738012122E39800D95
:0D195200122F128008122FEB80031230C4F8
:0F27B90002194B02194D02195202195702195CED
:10195F00900029E090007BF0E568900058F0E56A70
:10196F00900063F0E56B900064F0E56C900075F00B
:10197F00E56790007DF0E56990007EF0E5669000E8
:10198F0081F0E565900082F090002AE090013BF035
:10199F0090002BE090013CF090002CE090013DF086
:1019AF00900041E0900091F0900042E0900092F0A2
:1019BF00900043E0900093F0900044E0900094F08A
:1019CF00900045E0900095F0900046E0900096F072
:1019DF00900047E0900097F0900048E0900098F05A
:1019EF00900033E090009AF0900034E090009BF06C
:1019FF00900035E090009CF0900036E090009DF054
:101A0F007400900083F0744A900126F07461900185
:101A1F0027F07474900128F07463900129F0746FAB
:101A2F0090012AF0742090012BF0745290012CF049
:101A3F00744590012DF0743590012EF07452900181
:101A4F002FF07430900130F07435900131F0744103
:101A5F00900132F07420900133F07435900134F01E
:101A6F00900415E0900455F0743A90074FF074FD10
:101A7F00900750F012008F900004E4F0A3F0900054
:101A8F00067475F0A37430F09000087475F0A374A9
:101A9F0030F0855859D2CA754C00D29C741B9000F7
:101AAF0023F0E556C394065005E551B55203021BCA
:101ABF0068C207E55175F040A4FFAEF09003231202
:101ACF00001EE030E003D38001C39210E55175F0A2
:101ADF0040A4FFAEF090032412001EE030E003D3C9
:101AEF008001C3920FE55175F040A4FFAEF0900353
:101AFF002512001EE030E003D38001C39212E5519E
:101B0F0075F040A4FFAEF090032612001EE030E007
:101B1F0003D38001C39211E55175F040A4FFAEF0DD
:101B2F0090032712001EE030E003D38001C3B340BF
:101B3F0008E5B54440F5B58006E5B554BFF5B58564
:101B4F005152AE29AF2A7405BE00039F5007E545D9
:101B5F00D3940550028002D292E55AD394034006E3
:101B6F00E551640460028002C212E556D394055019
:101B7F0003021D45C207E551D394015003021C46D1
:101B8F00E55175F040A4FFAEF090031F12001EE068
:101B9F00A829B80007D3952A40021551E55165527F
:101BAF007003021C43E55175F040A4FFAEF09003A3
:101BBF002312001EE030E003D38001C39210E551E1
:101BCF0075F040A4FFAEF090032412001EE030E049
:101BDF0003D38001C3920FE55175F040A4FFAEF01F
:101BEF0090032512001EE030E003D38001C3921250
:101BFF00E55175F040A4FFAEF090032612001EE0F1
:101C0F0030E003D38001C39211E55175F040A4FF7A
:101C1F00AEF090032712001EE030E003D38001C323
:101C2F00B34008E5B54440F5B58006E5B554BFF5BA
:101C3F00B5855152021D45E556B406509000ADE0F2
:101C4F0030E003D38001C392109000AEE030E00388
:101C5F00D38001C3920F9000AFE030E003D3800137
:101C6F00C392129000B0E030E003D38001C3921111
:101C7F009000B1E030E003D38001C3B34008E5B575
:101C8F004440F5B58006E5B554BFF5B5E556B40744
:101C9F00509000A6E030E003D38001C39210900073
:101CAF00A7E030E003D38001C3920F9000A8E0308B
:101CBF00E003D38001C392129000A9E030E003D378
:101CCF008001C392119000AAE030E003D38001C3DA
:101CDF00B34008E5B54440F5B58006E5B554BFF50A
:101CEF00B5E556B4085090009FE030E003D3800173
:101CFF00C392109000A0E030E003D38001C3920F95
:101D0F009000A1E030E003D38001C392129000A2B3
:101D1F00E030E003D38001C392119000A3E030E0E4
:101D2F0003D38001C3B34008E5B54440F5B5800641
:101D3F00E5B554BFF5B5900073E07003021DDBE508
:101D4F005AD394044005A208B340028027E5457595
:101D5F00F00284FF7E0090014F12001EE0F55CE55B
:101D6F005CD3940F4009E55CC3940FF55C80037559
:101D7F005C008012E54575F00284FF7E0090014FF4
:101D8F0012001EE0F55CE54775F00A84FF7E0090B7
:101D9F00024F12001EE0F55FE55C255FD3946440AF
:101DAF000BE55C255FC39464F55C8003755C00E50F
:101DBF005C75F00284FF7E008F5CEFC39433500795
:101DCF00EF24CDF55C8003755CFF805FE55AD394FB
:101DDF00044005A208B340028035E54575F0028442
:101DEF00FF7E0090014F12001EE0F55CE55CD3947E
:101DFF000F4009E55CC3940FF55C8003755C00E54B
:101E0F005C75F00284FF7E00EF24CDF55C801CE54D
:101E1F004575F00284FF7E0090014F12001EE075A1
:101E2F00F00284FF7E00EF24CDF55CE595C394EBC3
:101E3F00400AC296C295C2A0C297801CA210B3409E
:101E4F0002D296A20FB34002D295A212B34002D291
:101E5F00A0A211B34002D297E562B40206E5516425
:101E6F000260028008E5B54440F5B58013E562B421
:101E7F000108E5B54440F5B58006E5B554BFF5B5A5
:101E8F00E595C3955C4004C2A28002D2A2E575D34A
:101E9F0094CD4007E575C394E940028004D20880D1
:101EAF0002C208A207B34005E556B407037575CD06
:101EBF00E595C395754004C2A18002D2A1E543C345
:101ECF00940640030224EDA2EDB350030224EDC2A9
:101EDF00EDE54360030220317E017F00E5BE124134
:101EEF00CFE5BD2FFF50010E900000EEF0A3EFF0F5
:101EFF00900029E0B401177E0F7FFF900000E0FCF7
:101F0F00A3E0FD120003900000EEF0A3EFF09000AD
:101F1F007AE0B4025B900000E0FEA3E0FF90000ABD
:101F2F00E0FCA3E0FDEDD39FEC9E400F900000E09E
:101F3F00F8A3E090000AC8F0A3C8F0900000E0FEFC
:101F4F00A3E0FF90000CE0FCA3E0FDEFD39DEE9C1F
:101F5F00400F900000E0F8A3E090000CC8F0A3C879
:101F6F00F0900000E0FEA3E0FF74041241C18F4423
:101F7F0090007AE07060900000E0FEA3E0FF900018
:101F8F000AE0FCA3E0FDEFD39DEE9C400D12000391
:101F9F00900000EEF0A3EFF08007900000E4F0A3B4
:101FAF00F0900000E0FEA3E0FF74101241CF90000C
:101FBF0026E08E048F05FF1241B1900000ECF0A3D4
:101FCF00EDF07400D39D74019C4008900001E0F582
:101FDF004480037544FFE54475F00AA4FFAEF07426
:101FEF00198E048F05FF1241B18D45ED2532FFAEDD
:101FFF003150010E74011241C18F45854532753143
:10200F0000EFD394624003754562900073E0640261
:10201F006006900067E060028005754301800375DC
:10202F00BB17E543B4010280030221217E017F002B
:10203F00E5BE1241CFE5BD2FFF50010E900000EE1F
:10204F00F0A3EFF0900073E0B4017EE53445336008
:10205F0025AC33AD341DBDFF011C8F028E038C06E2
:10206F008D07903BC512002EE493FE740193FFEF92
:10207F00C39AEE9B4002800578331241F9AE33AF1D
:10208F003474B3BE0025D39F4021900000E0FCA321
:10209F00E0FD0FBF00010E903BC512002EE493FE32
:1020AF00740193FFEDC39FEC9E40028005783312BD
:1020BF00003FAE33AF34E56C1241CF74648E048FA2
:1020CF0005FF1241B18D478033900067E0602D907E
:1020DF000000E0FEA3E0FFEFD39400EE9408400F62
:1020EF00900067E0B40104C20A8002D20A800D900A
:1020FF000067E0B40104D20A8002C20A900073E0C4
:10210F0064026006900067E0600575BB168003757A
:10211F004302E543B40202800302220F7E017F00D7
:10212F00E5BE1241CFE5BD2FFF50010E900000EE2E
:10213F00F0A3EFF0900073E0B4027EE53445336016
:10214F0025AC33AD341DBDFF011C8F028E038C06F1
:10215F008D07903E9912002EE493FE740193FFEFCA
:10216F00C39AEE9B4002800578331241F9AE33AF2C
:10217F003474B3BE0025D39F4021900000E0FCA330
:10218F00E0FD0FBF00010E903E9912002EE493FE6A
:10219F00740193FFEDC39FEC9E40028005783312CC
:1021AF00003FAE33AF34E56C1241CF74648E048FB1
:1021BF0005FF1241B18D478033900067E0602D908D
:1021CF000000E0FEA3E0FFEFD39400EE9408400F71
:1021DF00900067E0B40104C20A8002D20A800D9019
:1021EF000067E0B40104D20A8002C20A900073E0D3
:1021FF007003754700900067E07002C20A75BB1F3D
:10220F00E543B403457E017F00E5BE1241CFE5BD36
:10221F002FFF50010E900000EEF0A3EFF0740912A3
:10222F0041CF74E68E048F05FF1241B18C418D4270
:10223F00E54A2DFD50010C74018C068D071241C12A
:10224F008E418F4285424A75BB19E543B404028023
:10225F00030223D57E017F00E5BE1241CFE5BD2FDE
:10226F00FF50010E900000EEF0A3EFF07404124146
:10227F00C18F4BE566B401028003022344756D00E4
:10228F00756D00E56DD394074003022331E56D9022
:10229F0000411241E7E0D3954B501AE56D90004194
:1022AF001241E7E0F404254BFEE56D900037124133
:1022BF00E7EEF08017E56D9000411241E7E0C3951E
:1022CF004BFEE56D9000371241E7EEF0E56DC394DC
:1022DF00044009900085E0C3956D503BE56D602982
:1022EF00E56D9000371241E7FEE0FFEE90003FE012
:1022FF00D39F4013E56D9000371241E7E090003F08
:10230F00F0E56D900040F0800E900037E090003FB8
:10231F00F07400900040F0786D740126F6400302CF
:10232F002292900040E0F4042408F556E556D39429
:10233F00054002C292E566D39401402FE54BD3943A
:10234F006E4004D2158002C215755605E566B402BB
:10235F0005A215B340028003755607E566B4030660
:10236F00A215B3B340028003755607E55765566053
:10237F0026E55104F552E556B4050BE557B40606AC
:10238F00E55164016002800C75510290004E74019A
:10239F00F0755A00855657E556B40708E5B54480E1
:1023AF00F5B58006E5B5547FF5B5E55664066005CD
:1023BF00E556B40808E5B54410F5B58006E5B55403
:1023CF00EFF5B575BB13E543B4050280030224E9AD
:1023DF007E017F00E5BE1241CFE5BD2FFF50010EFC
:1023EF00900000EEF0A3EFF074041241C18F46E5A8
:1023FF0065B4020280030224E6756D00756D00E579
:10240F006DD39403400302249DE56D900033124178
:10241F00E7E0D39546501AE56D9000331241E7E09F
:10242F00F4042546FEE56D90002D1241E7EEF08095
:10243F0017E56D9000331241E7E0C39546FEE56D59
:10244F0090002D1241E7EEF0E56D6029E56D9000EB
:10245F002D1241E7FEE0FFEE900031E0D39F4013D5
:10246F00E56D90002D1241E7E0900031F0E56D90A1
:10247F000032F0800E90002DE0900031F07400904B
:10248F000032F0786D740126F6400302240E90009E
:10249F0083E07043E52A45296036E558C39403501D
:1024AF000A900032E004C394034002800790003288
:1024BF00E004F558E558D39402400A900032E00446
:1024CF00D3940250028007900032E004F558800741
:1024DF00900032E004F55875BB180543D2ECE56067
:1024EF00D39404500302266175CF01C2A2AE35AF5B
:1024FF00367488D39F74139E4005A2A5B34014AEC3
:10250F0035AF367488D39F74139E4005A2A4B34091
:10251F00028048783512003FAE35AF36EFB4883BB6
:10252F00EEB41337A2A5B35009900050E0D39551E4
:10253F005002800405518011A2A5B350089000509D
:10254F00E0655160028002D207A2A4B35007E551A3
:10255F00D39401500280041551C207A2A5B3B35002
:10256F0006A2A4B3B340028006753600753500E5A8
:10257F005165527003022618E55175F040A4FFAE65
:10258F00F090032312001EE030E003D38001C392CA
:10259F0010E55175F040A4FFAEF090032412001E19
:1025AF00E030E003D38001C3920FE55175F040A4F2
:1025BF00FFAEF090032512001EE030E003D3800140
:1025CF00C39212E55175F040A4FFAEF090032612AE
:1025DF00001EE030E003D38001C39211E55175F086
:1025EF0040A4FFAEF090032712001EE030E003D3AB
:1025FF008001C3B34008E5B54440F5B58006E5B5A5
:10260F0054BFF5B5C2A1855152E595C3955D400AFA
:10261F00C296C295C2A0C297801CA210B34002D22C
:10262F0096A20FB34002D295A212B34002D2A0A23B
:10263F0011B34002D297A20740057575CD8003757F
:10264F0075FFE595C395754004C2A18002D2A10222
:10265F0024F7A214B3500DAE25AF2674E8C39F74B0
:10266F00039E4002800B75FFA0D214E5B554FBF515
:10267F00B5AE25AF26EFD39420EE944E500302272C
:10268F007B120471C28E758D00758B00754C00D254
:10269F008EC2077574007573007575CD755105750C
:1026AF002400752300755400755A00C28790005A94
:1026BF00E06004D2908002C29090004AE0B401041E
:1026CF00D2948002C294900049E0B40104D2938066
:1026DF0002C293A20AB34004D2918002C291900029
:1026EF006CE0601812384EA200B34008E5B54408FC
:1026FF00F5B58006E5B554F7F5B58002C200900038
:10270F006FE060181239A3A202B34008E5B5440286
:10271F00F5B58006E5B554FDF5B58006E5B554FD74
:10272F00F5B590000E74FDF0A374E8F0E543B40620
:10273F0003754300900025E4F0752600752500759C
:10274F008D00758B00754C00900024E0C3940350EE
:10275F0008900024E004F080067403900024F090A9
:10276F000024E0B40306E5B554FEF5B5AE27AF2857
:10277F00EFD39410EE9427401CC2CA75CD0075CCD0
:10278F0000752800752700D2CA754E00752A00758E
:08279F002900755500020AF83B
:103B55000000010001320164019601960200021283
:103B650002240200020003000340038003C0040096
:103B75000440048004C00500060006000600060097
:103B8500060006000600060000FF013101630195ED
:103B950001FF01FF0211022302FF02FF02FF033FA3
:103BA500037F03BF03FF043F047F04BF04FF05FF3A
:103BB50006FF06FF06FF06FF06FF06FF06FF06FFD8
:103BC5000FAA0FA50F9F0F9A0F940F8D0F870F80C8
:103BD5000F780F710F680F600F570F4E0F450F3B92
:103BE5000F300F250F1A0F0E0F020EF50EE80EDB24
:103BF5000ECC0EBE0EAE0E9F0E8E0E7D0E6C0E5AA8
:103C05000E470E340E200E0C0DF70DE20DCB0DB543
:103C15000D9D0D850D6D0D540D3A0D200D050CE90D
:103C25000CCE0CB10C940C760C580C3A0C1B0BFBFF
:103C35000BDB0BBB0B9A0B790B570B350B130AF1EF
:103C45000ACE0AAB0A870A640A400A1C09F809D495
:103C550009B0098C09670943091F08FB08D608B292
:103C6500088E086A0846082307FF07DC07B9079688
:103C750007730751072F070D06EC06CA06AA068922
:103C850006690649062A060A05EC05CD05B0059222
:103C950005750558053C0520050504EA04CF04B55E
:103CA500049C04820469045104390422040B03F4BE
:103CB50003DE03C803B2039D038903750361034D46
:103CC500033B03280316030402F202E102D102C0FA
:103CD50002B002A0029102820273026502570249F4
:103CE500023C022F02220216020901FD01F201E641
:103CF50001DB01D001C601BB01B101A7019D019402
:103D0500018B018201790170016801600158015040
:103D15000148014101390132012B0125011E01181C
:103D25000111010B010500FF00FA0FA60FA00F9965
:103D35000F920F8B0F840F7C0F740F6B0F620F5850
:103D45000F4E0F430F380F2C0F1F0F120F050EF7D5
:103D55000EE80ED80EC80EB70EA50E930E800E6C8B
:103D65000E580E420E2C0E150DFD0DE40DCB0DB1AA
:103D75000D950D790D5D0D3F0D200D010CE10CC06C
:103D85000C9E0C7C0C590C350C100BEA0BC40B9ECD
:103D95000B760B4F0B260AFD0AD40AAA0A800A5590
:103DA5000A2A09FF09D409A8097C0950092508F937
:103DB50008CD08A10875084A081E07F307C8079D1E
:103DC50007730749072006F706CE06A6067E06579F
:103DD5000630060A05E405BF059B0577055405323F
:103DE500051004EF04CE04AE048F047104530435AA
:103DF500041903FD03E203C703AD0394037B0363C7
:103E0500034B0334031E030802F302DE02CA02B6A3
:103E150002A30291027F026D025C024C023C022C5D
:103E2500021D020E020001F201E401D701CA01BE22
:103E350001B101A6019A018F0185017A0170016620
:103E4500015D0153014A0141013901310129012176
:103E550001190112010B010400FD00F700F000EA51
:103E650000E400DE00D900D300CE00C900C400BFC5
:103E750000BA00B500B100AD00A800A400A0009CE8
:103E8500009900950091008E008A008700840081CA
:043E9500007E007B30
:1027C800751A00751900AE19AF1AAC17AD18EDC31C
:1027D8009FEC9E401674FF1241A175CF01781A74C0
:1027E8000126F6500418E436F650DB22900787E4F9
:1027F800F0A3F0751000750F00751300751400C272
:1028080016D21722C2AF75D900758F0375B7A57593
:10281800B7F190F800E4F0758F0175B7A575B7F1B9
:10282800E50890F800F075B7A575B7F190F801E4E0
:10283800F075B7A575B7F190079EE090F802F075AE
:10284800B7A575B7F19007A2E090F803F075B7A5A2
:1028580075B7F190079FE090F804F075B7A575B7C4
:10286800F19007A0E090F805F075B7A575B7F1905D
:1028780007A1E090F806F075B7A575B7F19007A322
:10288800E090F807F0758F0075D940D2AF22900715
:1028980089E0B4AB61C2AF75D90075B62275F5226F
:1028A800758F0375B7A575B7F1740090F600F075CC
:1028B8008F01750A00750900AE09AF0A7413BE00CE
:1028C800279F402475B7A575B7F190078A12001E97
:1028D800E0FC90F60012001EECF0780A740126F66F
:1028E800500418E436F650D0758F0075F51175B69A
:1028F8002075D940D2AF22C2AF75D90075F52275BF
:102908000A00750900AE09AF0A7413BE00229F4081
:102918001F90F60012001EE493FC90078A12001E16
:10292800ECF0780A740126F6500418E436F650D50F
:1029380075F51175D940D2AF22900789E0B4AA0283
:102948008003022A7EC2AF75D90075B62275F522BA
:10295800758F0375B7A575B7F1740090EE00F07523
:10296800B7A575B7F1740090F000F075B7A575B705
:10297800F1740090F200F075B7A575B7F174009086
:10298800F400F0758F01750A00750900AE09AF0AE9
:1029980074FFC39F74019E402475B7A575B7F19065
:1029A800004F12001EE0FC90EE0012001EECF078C2
:1029B8000A740126F6500418E436F650CF750A005A
:1029C800750900AE09AF0A74FFC39F74019E4024C5
:1029D80075B7A575B7F190024F12001EE0FC90F094
:1029E8000012001EECF0780A740126F6500418E470
:1029F80036F650CF750A00750900AE09AF0A74FFA4
:102A0800C39F74019E402475B7A575B7F190044F14
:102A180012001EE0FC90F20012001EECF0780A741E
:102A28000126F6500418E436F650CF750A007509E9
:102A380000AE09AF0A74FFC39F74019E402475B7A6
:102A4800A575B7F190064F12001EE0FC90F4001235
:102A5800001EECF0780A740126F6500418E436F6E5
:102A680050CF758F0075F51175B62075D940D2AF66
:102A7800743A90074FF022900789E0B4AA028003C5
:102A8800022BBCC2AF75D90075B62275F522758FB9
:102A98000375B7A575B7F1740090E600F075B7A592
:102AA80075B7F1740090E800F075B7A575B7F174C3
:102AB8000090EA00F075B7A575B7F1740090EC00C6
:102AC800F0758F01750A00750900AE09AF0A74FF29
:102AD800C39F74019E402475B7A575B7F190004F48
:102AE80012001EE0FC90E60012001EECF0780A745A
:102AF8000126F6500418E436F650CF750A00750919
:102B080000AE09AF0A74FFC39F74019E402475B7D5
:102B1800A575B7F190024F12001EE0FC90E8001274
:102B2800001EECF0780A740126F6500418E436F614
:102B380050CF750A00750900AE09AF0A74FFC39F2C
:102B480074019E402475B7A575B7F190044F120023
:102B58001EE0FC90EA0012001EECF0780A740126D0
:102B6800F6500418E436F650CF750A00750900AE21
:102B780009AF0A74FFC39F74019E402475B7A575F9
:102B8800B7F190064F12001EE0FC90EC0012001EF8
:102B9800ECF0780A740126F6500418E436F650CFA3
:102BA800758F0075F51175B62075D940D2AF743A96
:102BB80090074FF022900789E0B4AA028003022C04
:102BC800FAC2AF75D90075B62275F522758F0375EF
:102BD800B7A575B7F1740090DE00F075B7A575B7A5
:102BE800F1740090E000F075B7A575B7F174009026
:102BF800E200F075B7A575B7F1740090E400F075C0
:102C08008F01750A00750900AE09AF0A74FFC39FEA
:102C180074019E402475B7A575B7F190004F120056
:102C28001EE0FC90DE0012001EECF0780A7401260B
:102C3800F6500418E436F650CF750A00750900AE50
:102C480009AF0A74FFC39F74019E402475B7A57528
:102C5800B7F190024F12001EE0FC90E00012001E37
:102C6800ECF0780A740126F6500418E436F650CFD2
:102C7800750A00750900AE09AF0A74FFC39F740195
:102C88009E402475B7A575B7F190044F12001EE059
:102C9800FC90E20012001EECF0780A740126F6504F
:102CA8000418E436F650CF750A00750900AE09AF6E
:102CB8000A74FFC39F74019E402475B7A575B7F1C8
:102CC80090064F12001EE0FC90E40012001EECF08B
:102CD800780A740126F6500418E436F650CF758F3A
:102CE8000075F51175B62075D940D2AF743A9007C2
:102CF8004FF022900789E0B4AA028003022E38C25E
:102D0800AF75D90075B62275F522758F0375B7A50D
:102D180075B7F1740090D600F075B7A575B7F17462
:102D28000090D800F075B7A575B7F1740090DA0077
:102D3800F075B7A575B7F1740090DC00F0758F01D8
:102D4800750A00750900AE09AF0A74FFC39F7401C4
:102D58009E402475B7A575B7F190004F12001EE08C
:102D6800FC90D60012001EECF0780A740126F6508A
:102D78000418E436F650CF750A00750900AE09AF9D
:102D88000A74FFC39F74019E402475B7A575B7F1F7
:102D980090024F12001EE0FC90D80012001EECF0CA
:102DA800780A740126F6500418E436F650CF750AEE
:102DB80000750900AE09AF0A74FFC39F74019E40F5
:102DC8002475B7A575B7F190044F12001EE0FC906A
:102DD800DA0012001EECF0780A740126F650041886
:102DE800E436F650CF750A00750900AE09AF0A74CB
:102DF800FFC39F74019E402475B7A575B7F190066F
:102E08004F12001EE0FC90DC0012001EECF0780A65
:102E1800740126F6500418E436F650CF758F007505
:102E2800F51175B62075D940D2AF743A90074FF0B6
:102E380022C2AF75D90075F522750A00750900AE72
:102E480009AF0A74FFC39F74019E401F90EE0012E1
:102E5800001EE493FC90004F12001EECF0780A74F8
:102E68000126F6500418E436F650D4750A007509A0
:102E780000AE09AF0A74FFC39F74019E401F90F013
:102E88000012001EE493FC90024F12001EECF07832
:102E98000A740126F6500418E436F650D4750A0070
:102EA800750900AE09AF0A74FFC39F74019E401FE5
:102EB80090F20012001EE493FC90044F12001EECE6
:102EC800F0780A740126F6500418E436F650D475E2
:102ED8000A00750900AE09AF0A74FFC39F74019E0A
:102EE800401F90F40012001EE493FC90064F12005D
:102EF8001EECF0780A740126F6500418E436F650F1
:102F0800D475F51175D940D2AF22C2AF75D9007505
:102F1800F522750A00750900AE09AF0A74FFC39F50
:102F280074019E401F90E60012001EE493FC90007E
:102F38004F12001EECF0780A740126F6500418E4CB
:102F480036F650D4750A00750900AE09AF0A74FF49
:102F5800C39F74019E401F90E80012001EE493FC7A
:102F680090024F12001EECF0780A740126F6500405
:102F780018E436F650D4750A00750900AE09AF0A90
:102F880074FFC39F74019E401F90EA0012001EE464
:102F980093FC90044F12001EECF0780A740126F698
:102FA800500418E436F650D4750A00750900AE09C5
:102FB800AF0A74FFC39F74019E401F90EC0012007B
:102FC8001EE493FC90064F12001EECF0780A740180
:102FD80026F6500418E436F650D475F51175D94024
:102FE800D2AF22C2AF75D90075F522750A007509EE
:102FF80000AE09AF0A74FFC39F74019E401F90DEA4
:103008000012001EE493FC90004F12001EECF078B2
:103018000A740126F6500418E436F650D4750A00EE
:10302800750900AE09AF0A74FFC39F74019E401F63
:1030380090E00012001EE493FC90024F12001EEC78
:10304800F0780A740126F6500418E436F650D47560
:103058000A00750900AE09AF0A74FFC39F74019E88
:10306800401F90E20012001EE493FC90044F1200EF
:103078001EECF0780A740126F6500418E436F6506F
:10308800D4750A00750900AE09AF0A74FFC39F74AE
:10309800019E401F90E40012001EE493FC90064F2E
:1030A80012001EECF0780A740126F6500418E43673
:1030B800F650D475F51175D940D2AF22C2AF75D983
:1030C8000075F522750A00750900AE09AF0A74FF8C
:1030D800C39F74019E401F90D60012001EE493FC0B
:1030E80090004F12001EECF0780A740126F6500486
:1030F80018E436F650D4750A00750900AE09AF0A0F
:1031080074FFC39F74019E401F90D80012001EE4F4
:1031180093FC90024F12001EECF0780A740126F618
:10312800500418E436F650D4750A00750900AE0943
:10313800AF0A74FFC39F74019E401F90DA0012000B
:103148001EE493FC90044F12001EECF0780A740100
:1031580026F6500418E436F650D4750A00750900AE
:10316800AE09AF0A74FFC39F74019E401F90DC0034
:1031780012001EE493FC90064F12001EECF0780A31
:10318800740126F6500418E436F650D475F5117516
:10319800D940D2AF22E51464046006E59964FF6063
:1031A800028031A2164004D2168027E51460087404
:1031B800E62514900023F0E513600874F0251390B9
:1031C8000023F0E514B4010280FE751400751300A5
:1031D800C2168002C216E514903AF8F828287375CA
:1031E8001400E599B4FF03751301E599B4FE03755E
:1031F8001302E599B4FD03751303E599B4FC03754F
:103208001304E599B4FA03751305E599B4FB06753B
:103218001401120471E599B4F906751404120471C5
:10322800E599D394E54007E599C394F040028016E8
:103238008599157514027E017F00E515C394E61281
:1032480041CF8E0D8F0E900787E4F0A3F0E599D358
:1032580094C44007E599C394E640028028859915EF
:1032680075140374E5C39515F50E750D00AE0DAF15
:103278000E903B5512002EE493F874019390078743
:10328800C8F0A3C8F0D29902370C900787E0FEA3D4
:10329800E0FFEFC39400EE94054009EFD394FFEEEE
:1032A80094064013900787E0FEA3E0FF90004F12BA
:1032B800001EE599F0800385996E90078712000E2D
:1032C800900787E0FEA3E0FFEFB40106EEB4070223
:1032D800800302351C90074FE0B43C02800302359E
:1032E8001CA20DB35005A20EB3400302340FC29CBA
:1032F80090007BE090078DF0900058E090078EF0EA
:10330800900063E090078FF0900064E0900790F0E1
:10331800900075E0900791F090007DE0900792F0A2
:1033280090007EE0900793F0900081E0900794F081
:10333800900082E0900795F090013BE0900796F0AE
:1033480090013CE0900797F090013DE0900798F0DD
:10335800900091E0900799F0900092E090079AF021
:10336800900093E090079BF0900094E090079CF009
:10337800900095E090079DF0900096E090079EF0F1
:10338800900097E090079FF0900098E09007A0F0D9
:1033980090009AE09007A1F090009BE09007A2F0BF
:1033A80090009CE09007A3F090009DE09007A4F0A7
:1033B8007400900083F012008F74AB900789F012AC
:0A33C800289674AA900789F0E558D2
:063AF8000231E7023292E8
:1033D200903B19F82828738012122941800D122A75
:0B33E2007F8008122BBD8003122CFB23
:0F3B19000233D90233DB0233E00233E50233EA31
:1033ED00900789E4F090013BE0700C90013CE07097
:1033FD000690013DE060028004C20D8002D20D02F4
:10340D003511C29C900079E090078AF090005FE042
:10341D0090078BF0900060E090078CF090007BE0BF
:10342D0090078DF0900058E090078EF0900063E0CB
:10343D0090078FF0900064E0900790F0900075E099
:10344D00900791F090007DE0900792F090007EE063
:10345D00900793F0900081E0900794F0900082E047
:10346D00900795F090013BE0900796F090013CE0BD
:10347D00900797F090013DE0900798F0900091E053
:10348D00900799F0900092E090079AF0900093E0E9
:10349D0090079BF0900094E090079CF0900095E0D1
:1034AD0090079DF0900096E090079EF0900097E0B9
:1034BD0090079FF0900098E09007A0F090009AE0A0
:1034CD009007A1F090009BE09007A2F090009CE087
:1034DD009007A3F090009DE09007A4F07400900079
:1034ED0083F074AB900789F012289674AA9007891F
:1034FD00F0122941122A7F122BBD122CFBD29C7582
:10350D0099FB80FED29C7514007513007599FB0212
:10351D00370C900787E0FEA3E0FFEF4E700685990C
:10352D0010750F00900787E0FEA3E0FF74016F4E4A
:10353D00701BAC0FAD10AA0DAB0EED2BFBEC3AFAD8
:10354D008A068B0790004F12001EE599F0900787B1
:10355D0012000E900787E0FEA3E0FF74026F4E701D
:10356D000C12008F85159975140075130002370C18
:10357D00900787E0FEA3E0FF90004F12001EE59933
:10358D00F090078712000E900787E0FEA3E0FFACD6
:10359D000DAD0E8F028E038C068D07903B8D1200A4
:1035AD002EE493F9740193FEEAD39EEB99400985BD
:1035BD00159975140075130002370C900787E0FEFE
:1035CD00A3E0FF90004F12001EE599F090078712BF
:1035DD00000E900787E0FEA3E0FFEFB40006EEB407
:1035ED000102800302370C90001CE0D394C7400BFE
:1035FD0090001CE0C394C8F516801A90001CE0D30F
:10360D009463400B90001CE0C39464F51680069003
:10361D00001CE0F516E51675F002A4FFAEF08F6DF7
:10362D00EF90004F1241E7EFFCE0FDEC90005212DD
:10363D0041E7EDFCE0FDEC2DB5160280030236FEF0
:10364D000FEF90004F1241E7E56DFFE0FCEF9000AA
:10365D00531241E7ECFFE0FCEFC39CB5160280036B
:10366D000236FEE56D9000511241E7E56DFFE0FC7D
:10367D00EF9000541241E7ECFFE0FCEF2CB5167112
:10368D00E56D9000551241E7E0C3951690079EF049
:10369D00E56D9000561241E7E0C3951690079FF037
:1036AD00E56D9000591241E7E0C395169007A0F023
:1036BD00E56D90005A1241E7E0C395169007A1F011
:1036CD00E56D90005B1241E7E0C395169007A2F0FF
:1036DD00E56D90005C1241E7E0C395169007A3F0ED
:1036ED0012280C7599F97518647517001227C88082
:0F36FD00FE7599FF7518647517001227C880FEB7
:093AFE0002351F02357D0235C8B6
:10370C0022E513903B07F828287302384D90078761
:10371C00E0FEA3E0FF90001212001EE0F599900766
:10372C008712000E900787E0FEA3E0FF74116F4E26
:10373C00700375130002384D85649902384D90075B
:10374C0087E0FEA3E0FF90004F12001EE0F599EF1A
:10375C00B40107EEB4070375130090078712000E2F
:07376C0002384D900788E0D0
:0F3B070002371602371902374402374A02376F66
:10377300903B28F8282873852499023842852A9992
:103783000238428544990238428547990238428576
:103793005199023842856299023842855699023816
:1037A3004285589902384275700090006AE07006AD
:1037B300900069E060028016A2A44006E57044040C
:1037C300F570A2A54006E5704402F570801A9000DA
:1037D3004AE0B40106E5704410F570900049E0B486
:1037E3000106E5704420F570A207B34006E5704476
:1037F30001F570A20AB34006E5704408F5708570C0
:1038030099803CA217B340077599FAC2178017A293
:1038130013B3400575990F800B900023E0F5999041
:103823000023E4F0C21380178542998012854B99D7
:0F383300800D85469980087599FC8003751300F8
:103B280002377A02378002378602378C02379202D0
:103B3800379802379E0237A40237AA02380602389D
:0D3B48002B02383002383502383A02383F7F
:0B38420090078712000E800312004860
:033B160002384A28
:10384D002290006CE0B4010385241190006CE0B46B
:10385D000203852A1190006CE0B403038544119096
:10386D00006CE0B4040385471190006CE0B40503CF
:10387D0085511190006CE0B4060385561190006CD3
:10388D00E0B4070385581190006DE0FE90006EE0E6
:10389D00C39E500302392490006CE0D39404402C55
:1038AD0090006DE0D39511500990006EE0C3951115
:1038BD0050028002D20090006DE0D3951150099016
:1038CD00006EE0C395115002C200804990006CE07B
:1038DD00B4041890006EE0C395115002D200900010
:1038ED006DE0D395114002C200802A90006DE0C3B7
:1038FD009511500990006EE0D3951150028002D2BF
:10390D000090006DE0D39511500990006EE0C395C5
:10391D00115002C200807E90006CE0D39404402CC4
:10392D0090006DE0C39511400990006EE0D39511A4
:10393D0040028002C20090006DE0C39511400990D5
:10394D00006EE0D395114002D200804990006CE0EA
:10395D00B4041890006DE0C395115002C2009000A0
:10396D006EE0D395114002D200802A90006DE0C325
:10397D009511400990006EE0D395114002D2009050
:10398D00006DE0D39511400990006EE0C395114094
:10399D00028002C2002290006FE0B4010385241161
:1039AD0090006FE0B40203852A1190006FE0B4031C
:1039BD000385441190006FE0B40403854711900016
:1039CD006FE0B4050385511190006FE0B4060385D7
:1039DD00561190006FE0B40703855811900070E008
:1039ED00FE900071E0C39E5003023A7990006FE0A3
:1039FD00D39404402C900070E0D3951150099000A1
:103A0D0071E0C3951150028002D202900070E0D394
:103A1D0095115009900071E0C395115002C20280BA
:103A2D004990006FE0B40418900071E0C3951150F7
:103A3D0002D202900070E0D395114002C202802A9A
:103A4D00900070E0C395115009900071E0D395116D
:103A5D0050028002D202900070E0D395115009906F
:103A6D000071E0C395115002C202807E90006FE09C
:103A7D00D39404402C900070E0C395114009900040
:103A8D0071E0D3951140028002C202900070E0C334
:103A9D0095114009900071E0D395114002D202803A
:103AAD004990006FE0B40418900070E0C395115078
:103ABD0002C202900071E0D395114002D202802A19
:103ACD00900070E0C395114009900071E0D39511FD
:103ADD004002D202900070E0D39511400990007120
:0B3AED00E0C3951140028002C20222DB
:0941E7002582F5825002058322B5
:10002E00EF2F500205832582F582E5833E2EF58360
:01003E00229F
:08000300C3EF9DFFEE9CFE22FD
:08003F000806B60002180622B3
:0D000E00A3E004F070061241DDE004F022D2
:0841F9000816B6FF0218162299
:0E41C100048007C3CE13CECF13CFD5E0F62275
:10406F00BC000FBE0008ED8FF084FFADF022E4FE20
:10407F00FF22BE000DEF60FE54F0606F20E70302D9
:10408F004125EAC0E0EBC0E078017A0075F001EE5F
:10409F0020E710EF25E0FFEE33FE0AC5F023C5F051
:1040AF0030E7F0EA5407F9096A7A007B00600108EB
:1040BF00C3EC9E40167004ED9F4010ED9FFDEC9EEB
:1040CF00FCE5F0CA4ACA03F5F08005E5F003F5F008
:1040DF00C3EE13FEEF13FFD9D77908CACBCAD8D0D6
:1040EF00EAFEEBFFD0E0FBD0E0FA22EC8FF084FC8D
:1040FF00ED54F045F0C48FF084FEEDC454F045F05C
:10410F00C48FF084FDEEC4FE54F02DFFEE540F3C2F
:10411F00FEADF07C0022790078008FF0EC7E082055
:10412F00E70DC3CD33CD33C933C9C833C8DEF084EF
:10413F0049F9E5F08FF0BE00E6FD7C00E9FFE8FEEF
:01414F00224D
:0E41CF00F88FF0A4FFE5F0CE88F0A42EFE22BB
:1041A100600D782B0241AB007830D8FED5E0F822C3
:1041B100EEC0E07E0012406FEFFDEEFCD0E0FE228B
:03000B000241505F
:03001B0002416B34
:03002B0002418609
:030000000241F0CA
:0941F00075817675D000020656B7
:0B001E00E5822FF582E5833EF583228A
:0A41DD000582D582021583158222A7
:10415000C0E0C0F0C083C082C0D075D00012064B52
:10416000D0D0D082D083D0F0D0E032C0E0C0F0C058
:1041700083C082C0D075D00012064ED0D0D082D07D
:1041800083D0F0D0E032C0E0C0F0C083C082C0D0A5
:1041900075D000120651D0D0D082D083D0F0D0E0BC
:0141A00032EC
:00000001FF
